:1000000010C0189518951895189518951895189565
:100010001895189518951895189518951895189578
:1000200018958FE181BD87E181BD8FE58DBFC0E46B
:10003000EEE04E2E82E08EBFD2E0F2E05F2EEEEFD9
:10004000F1E0A0E6B0E088278D933197E9F76624C8
:100050008FEF87BB8FEF88BB8FEF81BB8FEF82BBAA
:10006000C29880E08093790080E08093630080E014
:100070008093680084EC8093760080E08093630036
:1000800080E08093680084EC8093760080E082BBFF
:10009000C09AC19AC59AC49AC298C39A84EF91E053
:1000A0006FD480E08093790080E090E1AAE6B0E030
:1000B0008D939C9380E090E0AEE6B0E08D939C93AE
:1000C00000917900003009F013C088E08093A4000B
:1000D00087E08093A50080E290E0ACE6B0E08D93ED
:1000E0009C9380E290E0A0E7B0E08D939C9312C0D7
:1000F00086E08093A40085E08093A50088E290E0EC
:10010000ACE6B0E08D939C9388E290E0A0E7B0E08D
:100110008D939C93C39884E690E032D4C39A6AD2BC
:1001200088E290E0A4E6B0E08D939C9388E090E0B4
:10013000A6E6B0E08D939C93A3E8B0E0E2EAF9E094
:1001400000D461D388E290E0A4E6B0E08D939C9364
:1001500080E190E0A6E6B0E08D939C93A3E8B0E048
:10016000E6EBF9E0EED34FD3E1E0F0E0FAD388E13B
:1001700090E0A6E6B0E08D939C9380E690E0A4E644
:10018000B0E08D939C93A3E8B0E0EAECF9E0D9D31A
:100190003AD380E290E0A4E6B0E08D939C9380E2B5
:1001A00090E0A6E6B0E08D939C93A3E8B0E0EEEC7F
:1001B000F9E0C7D328D38FEF8093740088E290E0F2
:1001C000A6E6B0E08D939C9380E090E0A4E6B0E0DA
:1001D0008D939C93A4E6B0E00D911C91003F50E0FC
:1001E000150710F009F00EC000D3A4E6B0E00D91A1
:1001F0001C9148E050E0040F151FA4E6B0E00D93F9
:100200001C93E8CF88E090E0A4E6B0E08D939C9347
:1002100080E390E0A6E6B0E08D939C93A3E8B0E085
:10022000E2EEF9E08ED3EFD2E8E0F0E09AD32AD202
:10023000E6EEF2E08E2E9F2E80E090E0A6E6B0E0A3
:100240008D939C93A6E6B0E00D911C910F3350E086
:10025000150710F009F02CC080E090E0A4E6B0E0B3
:100260008D939C93A4E6B0E00D911C910F3350E068
:10027000150710F009F017C0E82DF92DA4E7B0E03C
:10028000C8950C9231968E2E9F2EAFD2A4E6B0E088
:100290000D911C9148E050E0040F151FA4E6B0E05A
:1002A0000D931C93DFCFA6E6B0E0F3D209F0CACFDE
:1002B00080EC8093760088E490E0A4E6B0E08D9333
:1002C0009C9388E190E0A6E6B0E08D939C93A3E830
:1002D000B0E0EEEFF9E035D396D2EAE0F0E041D3BA
:1002E0001ECFF894FFCF0000000004800000000043
:1002F0000008C0600000000000205EB000000000A8
:10030000043400EC0000000000C409BE000000003E
:100310000C01FFFF000000001C007EBF80000000F9
:100320002801E197800000007D1E84DFC0000001ED
:100330007EFF11EFC0000001CA7E8FEFE0000003D6
:10034000297038FFF80000061004407D0800000303
:1003500083D002787C00000721009CF7040000078E
:10036000910030F9BE00000765BEF8EDC600000739
:10037000B3FBE8EFFE000007F8FFF7E30E00000F05
:10038000F5E7E801FE00000F72800000FF00000F9B
:10039000F08000003E00000F608000007E00000E34
:1003A000E00000000600000E200000001600001C07
:1003B000000000000E00001C000000001E00001CD9
:1003C000000000001E00003C000000001A00002C8D
:1003D00000000000060001AC000000002E0001CC6F
:1003E00006700000360002B800F800001E00010C84
:1003F000018000FE0E00012C0FFC01F61E00008C97
:100400001F9203600F4001B803CA07FC1C00002CB8
:1004100001B809AE09C000EC04000BC41600006C62
:10042000000010781400004C000010801E40001CDA
:100430000000007019800004000000001A00000095
:10044000000000000F000018000000003A0000004B
:100450000000200022000000000C2800040000041E
:100460000043D00048000000038000005800000254
:10047000000001004000000201C000808000000078
:10048000007E12808000000100385E010000000044
:100490008040300100000000C02FE002000000009A
:1004A0006010100400000000100820080000000088
:1004B0000807C01000000000040000400000000019
:1004C00002000100000000000080060000000000A3
:1004D0000040080000000000003030000000000074
:1004E00000038000000020D0A1E6B0E08C9182BB28
:1004F000C498C19AC598C098C09AC59A15D0A0E66C
:10050000B0E08C9182BBC498C19AC598C098C09A3B
:10051000C59A0AD0A2E6B0E08C9182BBC19AC59878
:10052000C098C09AC59A0895C59A80E081BBC49AC4
:10053000C09AC598C19800B343E00423A0E8B0E096
:100540000C9300918000033009F401C0EDCFC19AF3
:10055000C59A8FEF81BB0895A6E6B0E00D911C917E
:1005600040E250E0DBD1AAE7B0E00D931C93A4E693
:10057000B0E00D911C91A4EAB0E04D915527B4D1A3
:10058000ACE7B0E04D935C93AAE7B0E00D911C910D
:10059000ACE7B0E04D915C91040F151FA2E7B0E00D
:1005A0000D931C93A2E7B0E00D911C91AAE6B0E078
:1005B0004D915C91040F151FA2E7B0E00D931C93C1
:1005C000A2E7B0E08D919C91A7E7B0E08D939C935A
:1005D000A2E7B0E011968C91A0E6B0E08C93A2E780
:1005E000B0E08C91A1E6B0E08C9384E2809362004D
:1005F0007ADF0895AAE6B0E011968C91A0E6B0E00B
:100600008C93AAE6B0E08C91A1E6B0E08C9382E4F2
:100610008093620068DFACE6B0E011968C91A0E6B2
:10062000B0E08C93ACE6B0E08C91A1E6B0E08C93A6
:1006300083E48093620057DFAEE6B0E011968C91C0
:10064000A0E6B0E08C93AEE6B0E08C91A1E6B0E01D
:100650008C9380E48093620046DFA0E7B0E01196BF
:100660008C91A0E6B0E08C93A0E7B0E08C91A1E67D
:10067000B0E08C9381E48093620035DF80E8809362
:10068000620047DF80E08093600080E0809361003B
:1006900084E28093620027DF88E98093620039DF7B
:1006A00081E08093680000916800003F10F009F03D
:1006B0001EC081E08093690000916900003410F051
:1006C00009F00EC080E08093600080EC80936200AF
:1006D00015DFA9E6B0E08C918F5F8C9309F0ECCF29
:1006E000A8E6B0E08C918F5F8C9309F0DCCF089581
:1006F000AEE6B0E011968C91A0E6B0E08C93AEE649
:10070000B0E08C91A1E6B0E08C9380E4809362002D
:10071000EADE0895A6E6B0E00D911C9148E050E0B5
:10072000E3D0AAE7B0E04D935C93AAE7B0E00D9167
:100730001C9140E250E0F2D0AAE7B0E00D931C9388
:10074000AAE7B0E00D911C91AEE6B0E04D915C914E
:10075000040F151FAAE7B0E00D931C93AAE7B0E0C1
:100760008D919C91A2E7B0E08D939C93A4E6B0E0BC
:100770000D911C91A4EAB0E04D915527B5D0AAE7A0
:10078000B0E04D935C93A2E7B0E00D911C91AAE715
:10079000B0E04D915C91040F151FA2E7B0E00D93FE
:1007A0001C93A2E7B0E011968C91A0E6B0E08C9388
:1007B000A2E7B0E08C91A1E6B0E08C9384E2809354
:1007C000620091DE08958FDE88E980936200A1DEE9
:1007D00008958EDF84E9809362009BDE089588DFB0
:1007E0008CE98093620095DE089582DFF2DFB4DE4B
:1007F0008091740080936000809176008093620005
:100800007DDEEDDF0895A3E8B0E0C5D0AEE7B0E04F
:100810008C9381E080937F0040917E0000917F0067
:10082000041710F009F028C080917F00E2E8F0E0A2
:10083000E80F8827F81F01E0A1E8B0E088D0A1E820
:10084000B0E08C91082F40E2041BA5E7B0E00C93C8
:1008500014D0A4E6B0E00D911C9148E050E0040FE4
:10086000151FA4E6B0E00D931C93AFE7B0E08C91A8
:100870008F5F8C9309F0D0CF08954CDF8091750085
:1008800080936000809176008093620037DEA7DF5E
:100890000895ED91FC913196FC93EE93089508D064
:1008A0003DD000FC10D0089503D01ED001F8F9CF40
:1008B0000024E89457FF02C009D0689400F80BD0D8
:1008C00010F80124089502D009D00895509540955C
:1008D0004F5F5F4F0895E89417FF089500951095B6
:1008E0000F5F1F4F68940895352F242FE894452BF0
:1008F00011F468940895512F402F0027112780E1AB
:10090000440F551F001F111F021B130B416018F4E9
:10091000020F131F4E7F8A9599F70895752F642F44
:1009200055274427FF93F1E1889405C010F4460F42
:10093000571F5695479517950795FA95B9F7FF9163
:100940000895C8950D9231960020D9F708958191A8
:100950008D930A9519F08823D1F7089588278D93F0
:10096000089588EE93E00CD03197D9F70895319728
:10097000F1F70895689462F80895E89462F808958C
:10098000EF93FF93E8EEF3E03197F1F70197D1F79A
:10099000FF91EF9108958FEF83959D919923E1F752
:1009A0000895546F73686962612054363936334351
:1009B000204C434400005769746820616E204174E4
:1009C0006D656C2038353335000062790000526166
:1009D0006E6A69742044696F6C2D434F4D50537992
:1009E00073007777772E636F6D70737973312E6331
:1009F0006F6D2F776F726B62656E6368000044697C
:100A000073706C61792061204269746D617021009E
:00000001FF
